:020000040000FA
:040000006A303A2800
:040004000034003490
:08000800A000030EA100831209
:1000100005191128831601178312B2308100B1012E
:100020002C2883160113831203140B190310A80D37
:10003000A90DAA0DAB0DAC0DAC16FF302C02031DA3
:100040002C28FA302B02031D2C2832152A08AF0069
:100050002908AE002808AD008B100B11210E83007B
:06006000A00E200E0900B5
:0C007400203084008001840A80300402E7
:10008000031C3C28512283160C30850587018312FE
:10009000850187010730990000309A0010308316DF
:1000A0008E008312603083168F0083120030831617
:1000B000910000008312C830831681008312313012
:1000C0009000003083168C00831210308B00BD1B13
:1000D0006F2885196F286400851D6B2885233D1CBA
:1000E00072280F2381018E018F010B118B100B10D1
:1000F0008C018B178A20321996202E22B40B882867
:10010000031085190314BA0DF0303A020319B8210F
:1001100024237A2864003310B10A311F9528AC01DA
:10012000AB01AA01A901A801B101080032110130F7
:10013000B7008B132030370783169B001C141A0856
:100140008312A4001030370783169B001C141A0872
:100150008312A300A6000230A606003037078316DC
:100160009B001C141A088312A200A7000130A706E6
:100170008B17331CC12822090339A200A309A40943
:10018000A50924082F02031DB22923082E02031DEE
:100190003B2922082D02031DB22901303702031D1D
:1001A000D8283D19D7283E18D8283E143F14762267
:1001B00002303702031DE3283D19E228BE18E32868
:1001C000BE143F147D2203303702031DEE283D1973
:1001D000ED283E19EE283E153F14842204303702E4
:1001E000031DF9283D19F828BE19F928BE153F143A
:1001F0008B2205303702031D04293D1903293E1ABD
:1002000004293E163F14922206303702031D0F299F
:100210003D190E29BE1A0F29BE163F149922073028
:100220003702031D1A293D1919293E1B1A293E17A9
:100230003F14A02208303702031D25293D19242927
:10024000BE1B2529BE173F14A72209303702031D04
:1002500030293D192F294218302942143F14AE226B
:100260000A303702031D3B293D193A29C2183B29A0
:10027000C2143F14B52226082E02031DB2292708F6
:100280002D02031DB22901303702031D4E293D19ED
:100290004D293E1C4E293E103F14BC22023037022D
:1002A000031D59293D195829BE1C5929BE103F1458
:1002B000C02203303702031D64293D1963293E1D06
:1002C00064293E113F14C42204303702031D6F29F4
:1002D0003D196E29BE1D6F29BE113F14C82205307D
:1002E0003702031D7A293D1979293E1E7A293E12CB
:1002F0003F14CC2206303702031D85293D1984297D
:10030000BE1E8529BE123F14D02207303702031DBE
:1003100090293D198F293E1F90293E133F14D42266
:1003200008303702031D9B293D199A29BE1F9B29BE
:10033000BE133F14D82209303702031DA6293D19E8
:10034000A529421CA62942103F14DC220A3037029C
:10035000031DB1293D19B029C21CB129C2103F1497
:10036000E022B229B70A0B30370203180800992897
:100370000130B600B400B500B70085018701B213A3
:100380000C238A20B40BD129031085190314BA0D4C
:10039000F0303A020319F929B50BD1299630B5008E
:1003A0000522321DC1293211331CDB292D090339E5
:1003B000AD00AE09AF092F1CC1292D083002031969
:1003C000C1292D08B0002E1EC1298B1320303707FC
:1003D000BC002F08BB003C2210303707BC002E08A1
:1003E000BB003C2200303707BC002D08BB003C227C
:1003F0008B1785018701B70AB6010130B5000B30B4
:100400003702031CC1290F230800013037020319EA
:10041000E422023037020319E822033037020319BD
:10042000EC22043037020319F02205303702031999
:10043000F422063037020319F82207303702031975
:10044000FC22083037020319002309303702031950
:1004500004230A3037020319082308003F1C080050
:100460003F101030BC003E08BB003C223030BC00C6
:100470004208BB003C2208008B133B0883161C1566
:100480009A0083123C0883169B0055309D00AA30C9
:100490009D009C1464009C184A2A1C1183128B171F
:1004A0000800831600309B001C141A088312BD003C
:1004B000831610309B001C141A0883123D18BE00CE
:1004C000831630309B001C141A0883123D18C2009A
:1004D000831620309B001C141A088312C1000130BF
:1004E000C11BC100C1080319C1000800051640085E
:1004F0004107D0000F08D1000800851640084107C9
:10050000D2000F08D3000800051440084107D400AA
:100510000F08D5000800851440084107D6000F08D1
:10052000D7000800871440084107D8000F08D900F9
:100530000800071540084107DA000F08DB00080033
:10054000071440084107DC000F08DD00080087168B
:1005500040084107DE000F08DF00080007164008CA
:100560004107CC000F08CD0008008715400841075F
:10057000CE000F08CF00080005128E018F01080081
:1005800085128E018F01080005108E018F01080071
:1005900085108E018F01080087108E018F010800E1
:1005A00007118E018F01080007108E018F010800CE
:1005B00087128E018F01080007128E018F0108003B
:1005C00087118E018F0108000508103A8500080088
:1005D0000508203A850008000508013A8500080052
:1005E0000508023A850008000708023A870008005B
:1005F0000708043A870008000708013A8700080046
:100600000708203A870008000708103A870008000A
:100610000708083A870008003E18051608003E182B
:100620000516BE1885163E190514BE1985143E1A06
:100630008714BE1A07153E1B0714BE1B87164218E7
:100640000716C218871508003D1D08005008400213
:10065000031D2F2B51080F02031C2F2B05125208CC
:100660004002031D382B53080F02031C382B851240
:1006700054084002031D412B55080F02031C412B57
:10068000051056084002031D4A2B57080F02031C91
:100690004A2B851058084002031D532B59080F029E
:1006A000031C532B87105A084002031D5C2B5B0868
:1006B0000F02031C5C2B07115C084002031D652B15
:1006C0005D080F02031C652B07105E084002031D26
:1006D0006E2B5F080F02031C6E2B87124C08400222
:1006E000031D772B4D080F02031C772B07124E08B2
:1006F0004002031D802B4F080F02031C802B871123
:100700000C1C08000C10C00A0800B601B401B501A9
:100710003D1C8D2BBD01BD14942BBD1C922BBD0126
:100720003D15942BBD013D143D08B6006400982B87
:10073000992B9A2B9B2B9C2BB51B0516B51F0512CD
:10074000B40B962BB50B962B0310B60CB608031DF5
:0E075000962B0030BC003D08BB003C22080088
:084000000900030007000100A4
:02400E00CC33B1
:10420000010078007A007C007E007B0079007F004E
:104210007D007A0078007E007C00FF00FF00FF0038
:104220000000F200F600FA00FE00F200F600FA00CC
:10423000FE00F200F600FA00FE00FF00FF00FF00A3
:10424000010005000500050005000900090009003E
:1042500009000D000D000D000D00FF00FF00FF0024
:104260000000FF00FF00FF00FF00FF00FF00FF0055
:10427000FF00FF00FF00FF00FF00FF00FF00FF0046
:10428000FF00FF00FF00FF00FF00FF00FF00FF0036
:10429000FF00FF00FF00FF00FF00FF00FF00FF0026
:1042A000FF00FF00FF00FF00FF00FF00FF00FF0016
:1042B000FF00FF00FF00FF00FF00FF00FF00FF0006
:1042C000FF00FF00FF00FF00FF00FF00FF00FF00F6
:1042D000FF00FF00FF00FF00FF00FF00FF00FF00E6
:1042E000FF00FF00FF00FF00FF00FF00FF00FF00D6
:1042F000FF00FF00FF00FF00FF00FF00FF00DD00E8
:00000001FF
